:100000009E0178289300061086118611831606102B
:10001000861186110F308605831213089E182E282C
:100020003A308D0098305F203330920042201330F8
:100030008D0088305F20422064305E204220643092
:100040005E2022309200422028302D200C302D20BE
:1000500006302D209E1413082E281E1492001E1CFC
:100060003C288611033C031C4128412007308D00A9
:10007000D0305F20031408001E14FE3C03197328BF
:1000800086151E1C1E1006140F3086051208F03946
:1000900086040610920E1E18422832305E20031489
:1000A00008008F018E00FF308E07031C8F07031C92
:1000B000732803308D00DF305F2053288D01E83E28
:1000C0008C008D09FC30031C68288C0703186528F8
:1000D0008C0764008D0F65280C186E288C1C722804
:1000E00000007228080083130313831264000800C1
:1000F000FE300220013002206830022065300220EC
:100100006C3002206C3002206F3002202030022040
:10011000773002206F300220723002206C300220D3
:100120006430022003308F00E8305220FE3002207D
:100130000130022068300220653002206C3002203D
:100140006C3002206F30022020300220413002202B
:100150006E300220643002207230022069300220AA
:0E0160007530022001308F00F43052207828D4
:02400E00F13F80
:00000001FF
